S01E00002E2E5C62696E5C6F70656E626C745F786D63343730302E7372656353
S3150800000000600020151200085B1200085D12000847
S315080000105F12000861120008631200080000000061
S315080000200000000000000000000000006512000843
S315080000306712000800000000691200086B12000829
S315080000406F12000871120008731200087512000872
S3150800005077120008791200087B1200087D12000842
S315080000607F120008000000000000000000000000E9
S31508000070811200080000000083120008851200089B
S3150800008087120008891200088B1200088D120008D2
S315080000908F120008911200089312000895120008A2
S315080000A097120008991200089B1200089D12000872
S315080000B09F120008A1120008A3120008A512000842
S315080000C0A7120008A9120008AB120008AD12000812
S315080000D0AF120008B1120008B3120008B5120008E2
S315080000E0B7120008B9120008BB120008BD120008B2
S315080000F0BF120008C1120008C3120008C512000882
S31508000100C7120008C9120008CB120008CD12000851
S31508000110CF120008D1120008D3120008D512000821
S31508000120D7120008D9120008DB120008DD120008F1
S31508000130DF120008E1120008E3120008E5120008C1
S31508000140E7120008E9120008EB120008ED12000891
S31508000150EF120008F1120008F3120008F512000861
S315080001600000000000000000000000000000000081
S31508000170F7120008F9120008FB120008FD12000821
S31508000180FF120008011300080313000805130008EE
S3150800019007130008091300080B1300080D130008BD
S315080001A00F1300081113000813130008151300088D
S315080001B017130008191300081B1300081D1300085D
S315080001C01F1300082113000823130008251300082D
S315080001D027130008291300082B1300080000000045
S315080001E02D1300082F1300083113000833130008D5
S315080001F0351300080000000037130008000000004F
S3150800020010B5054C237833B9044B13B10448AFF342
S3150800021000800123237010BD80000020000000002C
S31508000220B81C0008084B10B51BB108490848AFF3BD
S3150800023000800848036803B910BD074B002BFBD0A4
S31508000240BDE81040184700BF0000000084000020E9
S31508000250B81C00086C00002000000000154B002B9D
S3150800026008BF134B9D46A3F5803A00218B460F46DF
S315080002701348144A121A01F053FC0F4B002B00D0F6
S3150800028098470E4B002B00D0984700200021040009
S315080002900D000D48002802D00C48AFF3008001F08D
S315080002A019FC2000290000F069FD01F0FFFB00BFE2
S315080002B000000800006000200000000000000000A8
S315080002C080000020900900200000000000000000C7
S315080002D008B500F045F8044B5B6A13F4005F01D1DA
S315080002E0002008BD012008BD008F024808B564201B
S315080002F000F006F808BD00BF08B500F007F808BD0D
S31508000300014B1880704700BFA000002008B501F017
S315080003105DF80F4B1B68984218D30E4B1B783BB9F8
S3150800032001220C4B1A704FF400720B4B5A6006E010
S315080003300022084B1A704FF00072074B5A6001F002
S3150800034045F8064B1B881844014B186008BD00BFCA
S315080003509C000020A200002000850248A000002082
S315080003604FF00072014B5A60704700BF0085024883
S3150800037082B00023019303E000BF019B0133019380
S31508000380019B8342F8D302B0704700BF72B60D4B8B
S315080003900D4A9A60BFF34F8F62B6D3F8882042F4AD
S315080003A07002C3F888205A6922F008025A61074980
S315080003B041F214028B5823F00F0343F004038B50C9
S315080003C0704700BF00ED00E000000008001000586C
S315080003D000487047001BB70010B51E4BDB6813F4C6
S315080003E0803F27D01C4BDB6813F0010F02D1FFF7C3
S315080003F0EFFF00E01948184B1B6813F0040F11D0E3
S3150800040015498A68C2F303628B68C3F306238C68AE
S31508000410C4F30644611C02FB0112B0FBF2F203FBB3
S31508000420022208E00C4B9B6803F07F030133B0FB04
S31508000430F3F200E0094A0749C868C0B20130B2FBC6
S31508000440F0F3086900F001000130B3FBF0F0044B4B
S31508000450186010BD004600501047005000366E0167
S315080004606C00002070B55F4B9A6842F04D029A60A6
S315080004704D22DA60A0331B6813F0010F09D15A4ADE
S31508000480536843F001035360574B1B6813F0010F81
S31508000490FAD0564B1B6813F4007F08D0534A93686A
S315080004A043F40073936041F64C50FFF761FF504CDC
S315080004B0636843F40023636040F6C410FFF758FFEF
S315080004C0636823F4803323F002036360494B5B6857
S315080004D013F0300F24D0103C636823F030036360B8
S315080004E0FFF776FF444BA3FB00231B0D013B626815
S315080004F042EA034363603E4BDA6822F00102DA609F
S315080005005A6822F400325A60394B1B6803F4607348
S31508000510B3F5607FF8D1334A936823F001039360FB
S31508000520334B5A6842F001025A605A6842F0100288
S315080005305A60324A9A605A6842F040025A605A68CB
S3150800054022F010025A605A6842F480225A60284BF8
S315080005501B6813F0040FFAD0254A536823F00103E9
S315080005605360234B1B6813F0010FFAD11D4A936899
S3150800057023F004039360224C4FF00113E360002636
S3150800058066612661266266620323E3611D4BA361E9
S315080005901D4BA362164D6B6823F040036B601B4B23
S315080005A0AB604FF41660FFF7E3FE194BAB604FF4F0
S315080005B06160FFF7DDFE174BAB604FF49650FFF70F
S315080005C0D7FE154BAB6041F27070FFF7D1FE134BA7
S315080005D0AB604FF4E150FFF7CBFE6660FFF7FCFE19
S315080005E070BD00BF604100500042005000440050FA
S315080005F010470050004700506BCA5F6B002F0B0175
S31508000600004600500500010003002001002F0501E7
S31508000610002F0301002F0201002F0101002F000106
S3150800062010B54FF00053044C0FCB84E80F00FFF7CA
S31508000630ADFEFFF717FF10BD700000205022014BDA
S315080006401A6070475455000C024B18600433196041
S31508000650704700BFF055000C10B4064AAA23136071
S31508000660552405490C60A021116003605DF8044B10
S31508000670704700BF5455000CA8AA000C30B4074BAD
S31508000680AA241C60064A5521116080251D601C603D
S3150800069011603023036030BC704700BF5455000C0E
S315080006A0A8AA000CF522014B1A6070475455000C95
S315080006B041F21003014AD058704700BF0010005895
S315080006C070B506460D46FFF7EDFFFFF7B7FF0024A6
S315080006D007E0631C55F8231055F82400FFF7B4FF0C
S315080006E002343F2CF5D93046FFF7B6FF70BD00BF80
S315080006F010B50446FFF7D6FF2046FFF7BFFF10BD2B
S31508000700F8B504460D461646624B98422FD003F5B7
S31508000710807398422BD003F58073984227D003F54F
S315080007208073984223D003F5807398421FD003F54F
S31508000730807398421BD003F58073984217D003F54F
S315080007408073984213D003F5807398420FD003F54F
S31508000750807398420BD003F5A063984207D003F53F
S315080007608073984203D043214B4800F00DFF33783D
S315080007701BB3082B23D0102B23D0182B23D0202BC8
S3150800078023D0282B23D0302B23D0382B23D0802BD3
S3150800079023D0882B23D0902B23D0982B23D0A02B83
S315080007A023D0C02B23D0C82B23D0D02B23D0D82B93
S315080007B023D0E02B23D1012322E0012320E00123CB
S315080007C01EE001231CE001231AE0012318E001239F
S315080007D016E0012314E0012312E0012310E00123AF
S315080007E00EE001230CE001230AE0012308E00123BF
S315080007F006E0012304E0012302E0012300E00023D0
S315080008001BB94421244800F0BFFEAB081F1D54F84D
S31508000810270005F00302D200F821914020EA0101E1
S3150800082044F82710606F6F000321B94020EA0101E0
S3150800083061671A498C4203D001F580718C4207D151
S31508000840216E012000FA05F521EA0505256617E05F
S315080008507168A9406160E908103154F8217005F003
S315080008600705AD000720A84027EA000044F8210044
S3150800087054F82170307A00FA05F53D4344F82150C2
S31508000880043354F82300317801FA02F2024344F89B
S315080008902320F8BD008002484C1B0008008E024841
S315080008A0020F20F07040034B53F8222013681843B8
S315080008B0106070477C1B0008034B1868034B5B6984
S315080008C003F00103D84070476C0000200046005032
S315080008D0020F20F07040034B53F822201368184388
S315080008E0106070476C1B000870B504460E46154626
S315080008F0494B98422FD003F5807398422BD003F5C5
S315080009008073984227D003F58073984223D003F565
S31508000910807398421FD003F5807398421BD003F565
S315080009208073984217D003F58073984213D003F565
S31508000930807398420FD003F5807398420BD003F565
S31508000940A063984207D003F58073984203D04321E9
S31508000950324800F019FE1DB3082D23D0102D23D0E0
S31508000960182D23D0202D23D0282D23D0302D23D069
S31508000970382D23D0802D23D0882D23D0902D23D019
S31508000980982D23D0A02D23D0C02D23D0C82D23D019
S31508000990D02D23D0D82D23D0E02D23D1012322E03A
S315080009A0012320E001231EE001231CE001231AE0B5
S315080009B0012318E0012316E0012314E0012312E0C5
S315080009C0012310E001230EE001230CE001230AE0D5
S315080009D0012308E0012306E0012304E0012302E0E5
S315080009E0012300E000231BB944210C4800F0CCFD8C
S315080009F0B308043354F8231006F00306F600F82269
S31508000A00B24021EA020244F8232054F82320B540D4
S31508000A10154344F8235070BD008002488C1B00081B
S31508000A2070B505460E4600F0FBF8F47904B91024B3
S31508000A3022463168284600F045F8B379013B640838
S31508000A400134240244EA430343F00103EB63337998
S31508000A50013B1B0643F481736B6373792BB16A6B95
S31508000A60013B42EA03436B6305E06A6B3379013B5A
S31508000A7042EA03436B634FF4A063AB634FF0FF3363
S31508000A80EB6433892B6470BDD0F8083113F0E06F3E
S31508000A9009D1836B13F0800FFBD14FF40053C36465
S31508000AA0C0F880107047C0F880117047D0F80C3134
S31508000AB013F0E06F02D1406D80B27047D0F81C0188
S31508000AC080B2704763293BD9002A3BD02DE9F04113
S31508000AD015460C460646FFF7EFFE1B49A1FB0037F5
S31508000AE07F09A1FB0431480940F2FF3E4FF0010C93
S31508000AF0E046714611E007FB01F300FB05F2B3FB84
S31508000B00F2F39C0AC3F30903B4F5806F04D29E4539
S31508000B1002D99E46A446884601390029EBD148F4F5
S31508000B20004333617269094B1340013D43EA85234B
S31508000B300CF1FF3C43EA0C4373610020BDE8F081E9
S31508000B4001207047012070471F85EB51EF8000FC9C
S31508000B5030B4D0F8084124F0E064C0F80841D0F871
S31508000B600851064C2C4041EA032343EA026244EA50
S31508000B700203C0F8083130BC704700BFC0C0FFF898
S31508000B8030B4D0F80C4124F0E064C0F80C41D0F839
S31508000B900C51074C2C4041EA032343EA026244EA1B
S31508000BA0020343F08053C0F80C3130BC704700BFD5
S31508000BB0C0C0FFEF10B5144B984208D14FF400603F
S31508000BC0FFF786FE4FF40060FFF76AFE10BD0F4B75
S31508000BD0984207D10E4C2046FFF77AFE2046FFF7CB
S31508000BE05FFE10BD0B4B984207D10B4C2046FFF712
S31508000BF06FFE2046FFF754FE10BD40F24B11074822
S31508000C0000F0C2FC10BD00BF0800034008000248FF
S31508000C10800000100840024800010010AC1B0008C4
S31508000C2010B504462F4B984205D003F50073984239
S31508000C3003D1012302E0012300E0002343B92A4B34
S31508000C409C4207D003F500739C4205D1012304E0BA
S31508000C50012302E0012300E0002343B9234B9C4211
S31508000C6007D003F500739C4205D1012304E0012354
S31508000C7002E0012300E000231BB951211C4800F0C3
S31508000C8083FC184B9C4203D003F500739C4203D1A6
S31508000C901848FFF78FFF19E0134B9C4203D003F562
S31508000CA000739C4203D11448FFF784FF0EE00F4BF4
S31508000CB09C4203D003F500739C4203D10F48FFF70B
S31508000CC079FF03E065210A4800F05EFC0323E36030
S31508000CD0E36813F0010FFBD0236C23F00F032364A2
S31508000CE010BD00BF00000340000002480040024853
S31508000CF0AC1B0008080003400800024808400248E8
S31508000D0010B5802209210748FFF7EEFD064C0022A0
S31508000D100D212046FFF7E8FD236E23F400532366D2
S31508000D2010BD00BF00850248008F024870B586B026
S31508000D3000238DF80C300126049602258DF81450F0
S31508000D400C4C03AA04212046FFF7DAFC90238DF801
S31508000D50003001968DF808506A4605212046FFF7AF
S31508000D60CFFC054AD36923F007033343D36106B0A2
S31508000D7070BD00BF008102480000034008B5FFF7B8
S31508000D80BFFF00F035FCFFF7D1FF00F03FFCFCE7A2
S31508000D9008B500F03BFA08BD10B500F0DDFAA0B1C1
S31508000DA0FFF796FA88B100F059FC00F0E7FA00F070
S31508000DB0D7FA20F0604020F07F00044B186000F05E
S31508000DC0CFFA446800F024FAA04710BD08ED00E009
S31508000DD070B508E0461C4D1C0B78037000F06CFCDF
S31508000DE0224630462946531E9CB2002AF2D170BDCF
S31508000DF0030E082B01D100F18060704738B505460F
S31508000E00002419E000F058FC04EB440293000C4A55
S31508000E10D358AB420ED804EB44018A0008490A4469
S31508000E20526813449D4205D204EB440083000B44E8
S31508000E30187A38BD0134E4B20E2CE3D9FF2038BD48
S31508000E40CC1B000838B50546002410E000F034FC39
S31508000E5004EB44029300084A13441B7AAB4204D1BC
S31508000E6004EB44018B00D05838BD0134E4B20E2C93
S31508000E70ECD94FF0FF3038BDCC1B000808B5C1F3DC
S31508000E80090353B90368994209D040F8041B4FF483
S31508000E908062FFF79DFF012008BD002008BD0120E4
S31508000EA008BD00BF2DE9F04106460068FFF7A6FF1A
S31508000EB0FF2833D000272CE000F0FEFB35683C0203
S31508000EC025443444043400F081FA00F10D08214623
S31508000ED02846FFF7F5FB05E000F078FA804520D3B1
S31508000EE000F0EAFBFFF7E4FB00F0010010F0FF0F4B
S31508000EF0F2D1FFF7DDFB30F0100315D1002305E032
S31508000F005A5DD2B2E15C8A4211D10133FF2BF7D97F
S31508000F100137032FD0D90120BDE8F0810020BDE8B4
S31508000F20F0810020BDE8F0810020BDE8F0810020B6
S31508000F30BDE8F08138B50D460B4B984207D00446FC
S31508000F400A4B994205D0FFF7ADFF18B908E0084CDF
S31508000F5000E0054C29462046FFF790FF10B938BD3A
S31508000F60002038BD204638BDA40000200040000CF3
S31508000F70A80400202DE9F04106460C4617461D46F2
S31508000F8021F47F7828F003080368B3F1FF3F04D102
S31508000F904146FFF773FF034630B33368984505D0DB
S31508000FA041463046FFF7C6FF0646D0B13368E41A15
S31508000FB03444043400F080FB331DE31AB3F5806F24
S31508000FC007D308F580613046FFF7B4FF064650B1EF
S31508000FD0041D17F8013B04F8013B013DEAD1012342
S31508000FE002E0002300E000231846BDE8F08100BFB8
S31508000FF0884230D8F8B505460E4670B30F2926D96B
S315080010002DE000F059FB2846FFF71CFF0746B0F114
S31508001010FF3F26D000F0DAF900F5CE5408343846FA
S31508001020FFF766FB05E000F0D1F984421BD300F018
S3150800103043FBFFF73DFB00F0010010F0FF0FF2D174
S31508001040FFF736FB30F020030FD10135EDB2B5427C
S31508001050D7D90120F8BD002070470020F8BD002030
S31508001060F8BD0020F8BD0020F8BD0020F8BD00BF7F
S315080010704FF0FF33024A1360024A1360704700BFFD
S31508001080A8040020A400002070B50D461646FFF7F8
S31508001090AFFE0446FFF7B2FEFF281AD060190138E2
S315080010A0FFF7ACFEFF2816D024F47F7323F0030362
S315080010B00A4A934206D12B46324621460848FFF78C
S315080010C059FF70BD2B46324621460648FFF752FFA8
S315080010D070BD002070BD002070BD00BF0040000C30
S315080010E0A4000020A804002070B50C46FFF780FE77
S315080010F00646FFF783FE054630190138FFF77EFEE0
S31508001100FF2D06D0FF2806D001462846FFF770FFB8
S3150800111070BD002070BD002070BD00BF114B1B685C
S31508001120B3F1FF3F18D000B583B00E4B59689A68E3
S315080011301144DA6811441A6911445A6911449A69C2
S315080011401144DA698B18DB4302AA42F8043D0421EC
S315080011500548FFF799FF01E00120704703B05DF8E5
S3150800116004FB00BFA40000200042000C0E4B1A68C6
S3150800117004331B6813440D4A126813440C4A126858
S3150800118013440C4A126813440B4A126813440B4A58
S3150800119012681344DB430A4A1268934201D10120BC
S315080011A070470020704700BF0040000C0840000C44
S315080011B00C40000C1040000C1440000C1840000CA9
S315080011C00042000C08B50D4B1B68B3F1FF3F04D075
S315080011D00A48FFF767FE034668B1094B1B68B3F177
S315080011E0FF3F05D00648FFF75DFE034610B902E04B
S315080011F0012300E00123184608BD00BFA400002013
S31508001200A8040020004870470040000C72B67047DA
S3150800121062B670470649074A074B9A42BEBF51F85D
S31508001220040B42F8040BF8E70448804704480047D3
S31508001230C41C0008000000206C00002021060008DD
S315080012405D0200083C493D4A002301E041F8043BA1
S315080012509142FBD3FFF792FDFEE7FEE7FEE7FEE7C6
S31508001260FEE7FEE7FEE7FEE7FEE7FEE7FEE7FEE748
S31508001270FEE7FEE7FEE7FEE7FEE7FEE7FEE7FEE738
S31508001280FEE7FEE7FEE7FEE7FEE7FEE7FEE7FEE728
S31508001290FEE7FEE7FEE7FEE7FEE7FEE7FEE7FEE718
S315080012A0FEE7FEE7FEE7FEE7FEE7FEE7FEE7FEE708
S315080012B0FEE7FEE7FEE7FEE7FEE7FEE7FEE7FEE7F8
S315080012C0FEE7FEE7FEE7FEE7FEE7FEE7FEE7FEE7E8
S315080012D0FEE7FEE7FEE7FEE7FEE7FEE7FEE7FEE7D8
S315080012E0FEE7FEE7FEE7FEE7FEE7FEE7FEE7FEE7C8
S315080012F0FEE7FEE7FEE7FEE7FEE7FEE7FEE7FEE7B8
S31508001300FEE7FEE7FEE7FEE7FEE7FEE7FEE7FEE7A7
S31508001310FEE7FEE7FEE7FEE7FEE7FEE7FEE7FEE797
S31508001320FEE7FEE7FEE7FEE7FEE7FEE7FEE7FEE787
S31508001330FEE7FEE7FEE7FEE78000002090090020B2
S3150800134008B5FFF795FE08BD08B5FFF79DFE08BD71
S3150800135008B5FFF7C9FE08BD08B5FFF707FF08BDC2
S3150800136008B5FFF74FFF08BD08B5FFF7D7FE0346D8
S3150800137010B1FFF727FF0346184608BD0022014BA8
S315080013801A60704710E000E008B5FFF7F7FF054B55
S31508001390054A5A6000229A6005211960034B1A60B3
S315080013A008BD00BF10E000E07F320200AC08002054
S315080013B0044B1B6813F4803F03D0034A13680133B8
S315080013C01360704710E000E0AC08002008B5FFF78E
S315080013D0EFFF014B186808BDAC08002008B50D4B97
S315080013E0D3F8143113F4805F12D101460948FFF788
S315080013F04BFB084BD3F8143113F4807FF9D0054A18
S31508001400D2F8183143F48073C2F81831012008BDA8
S31508001410002008BD00000340074BD3F8143113F031
S31508001420080F07D110B504460348FFF73FFB2070A5
S31508001430012010BD0020704700000340F0B585B0BC
S315080014404FF46143019308238DF808308DF809306D
S3150800145001258DF80A5010278DF80B700026ADF877
S315080014600C600C4C01A92046FFF7DAFA2B46042239
S3150800147039462046FFF76CFB2B46042231462046A8
S31508001480FFF77EFB236C23F00F0343F0020323646C
S3150800149005B0F0BD0000034070B506460D4640296C
S315080014A003D972210F4800F06FF82846FFF796FF18
S315080014B0012803D076210B4800F066F800240CE0DA
S315080014C000F0FAF8305DFFF789FF012803D07F2185
S315080014D0044800F059F80134A4B2ABB29C42EFD3E9
S315080014E070BD00BF801C000838B5224B1C789CB91B
S315080014F02148FFF791FF01283AD11F4B1B78002B93
S3150800150031D0FFF763FF1D4B186000221C4B1A7081
S315080015100122184B1A702BE00546194B1B7801332C
S3150800152015481844FFF778FF0446012810D1144BD4
S315080015301A780132D2B21A700F4B1B789A4214D11C
S3150800154010492846FFF744FC00220A4B1A700FE0A0
S31508001550FFF73CFF094B1B686433984207D9002400
S31508001560044B1C7004E01C4602E0002400E0002442
S31508001570204638BDF2080020B0080020F4080020F4
S31508001580F1080020B108002008B5024B196000F0E8
S3150800159093F8FCE7F808002008B500F085F801285C
S315080015A010D0094B1B78012B0CD1FFF70FFF074B07
S315080015B01B6803F5FA73984204D30022024B1A708B
S315080015C0FFF7EAFB08BD00BFFC0800200009002061
S315080015D008B50122044B1A70FFF7F8FE034B186092
S315080015E0FFF7DAFF08BD00BFFC080020000900204D
S315080015F008B5FFF7CDFB00F05BF8FFF7C5FEFFF770
S315080016009FFE00F00DF8FFF7E3FF08BD08B500F0F0
S3150800161053F8FFF7CDFE00F00FF8FFF7BDFF08BD42
S3150800162008B500F0B5F9FFF709FF0022014B1A705B
S3150800163008BD00BF0000002008B50648FFF754FFA4
S31508001640012805D10022044B1A70024800F0BEF9A1
S3150800165008BD00BF0409002000000020704700BF35
S3150800166008B5044B1B7813B9C9B2FFF715FF00F08C
S31508001670A5F908BD00000020044B1B78013B022B8E
S3150800168001D9402070470020704700BF00000020A5
S31508001690044B1B78013B022B01D9402070470020E0
S315080016A0704700BF0000002008B500F07FF908BDAC
S315080016B008B5FEF71BFE08BD08B5FEF71DFE08BDFA
S315080016C010B4002304E010F8011B0B44DBB22146DA
S315080016D04C1E0029F7D1136001205DF8044B7047B2
S315080016E00022014B5A70704744090020034BFE2222
S315080016F0DA7018710222A3F84420704744090020C2
S3150800170010B5054C00232370FFF7EAFFFF23E370AB
S315080017100123A4F8443010BD44090020064BFF22DB
S31508001720DA7000221A71597859719A71DA711A7237
S315080017300622A3F8442070474409002008B5002073
S31508001740FFF7D4FF08BD00BF084BFF22DA70084A2E
S315080017509A6400221A715A719A710721D9711A72FC
S315080017605A729A720822A3F8442070474409002046
S31508001770A81C0008044BFF22DA7042689A6401220A
S31508001780A3F84420704700BF4409002010B5084C50
S31508001790FF23E370E21D4168A06CFFF791FF2071FB
S315080017A000236371A3710823A4F8443010BD00BF59
S315080017B04409002008B53120FFF798FF08BD00BF8F
S315080017C038B5084CFF23E370002525716571FFF7CE
S315080017D053FFA071E571257265720723A4F844309A
S315080017E038BD00BF4409002038B5FFF779FF0D4C16
S315080017F001252570FF23E3701023237100236371ED
S31508001800FFF73AFFA071FFF743FFE071FFF740FFCC
S31508001810C0F3072020726572A5720823A4F8443025
S3150800182038BD00BF4409002038B505464478FFF79F
S3150800183023FF0138844203DD2220FFF757FF38BD16
S31508001840084C6A78A16C201DFFF7C2FAFF23E370E3
S315080018506B78A26C1344A3646B780133A4F8443004
S3150800186038BD00BF4409002038B504464578FFF75F
S3150800187003FF0138854203DD2220FFF737FF38BD15
S315080018806168084DA9646278281DFFF7A1FAFF234D
S31508001890EB706378AA6C1344AB6463780133A5F8DC
S315080018A0443038BD4409002038B505460D4B9C6CBC
S315080018B0FFF7E2FE6A1C411E2046FFF745FD18B9F0
S315080018C03120FFF713FF38BD064CFF23E370FFF7FF
S315080018D0D3FE0138A36C1844A0640123A4F844304D
S315080018E038BD00BF4409002038B504464578FFF7DF
S315080018F0C3FE0238854203DD2220FFF7F7FE38BD16
S315080019000F4BFF22DA700122A3F84420617831B91F
S31508001910FFF72AFD90B93120FFF7E8FE38BDA21C73
S31508001920074B986CFFF710FD18B93120FFF7DEFE5C
S3150800193038BD6378024A916C0B44936438BD00BF86
S315080019404409002008B54168074B986CFFF700FD6D
S3150800195018B93120FFF7CAFE08BD034BFF22DA701B
S315080019600122A3F8442008BD4409002008B5FFF762
S3150800197013FA034BFF22DA700122A3F8442008BDAC
S315080019804409002008B589B2FFF76AFE08BD00BF02
S31508001990054B00221A709A6483F84320A3F8442062
S315080019A09A705A70704700BF44090020024B187895
S315080019B000B10120704700BF440900200022024BF5
S315080019C083F84320704700BF4409002008B5037810
S315080019D0FF2B02D1FFF708FF50E0334A1278012A9D
S315080019E060D1C93B352B46D8DFE803F0334545427D
S315080019F045453F363C3945454545454545454545B3
S31508001A004545454545454545454545454545454578
S31508001A10454545454545241E1B2145454527452A37
S31508001A202D30FFF701FF29E0FFF71EFF26E0FFF73D
S31508001A30A1FE23E0FFF7AAFE20E0FFF785FE1DE0E2
S31508001A40FFF77CFE1AE0FFF769FE17E0FFF758FE7E
S31508001A5014E0FFF729FF11E0FFF746FF0EE0FFF756
S31508001A60AFFE0BE0FFF76EFF08E0FFF77FFF05E02C
S31508001A70FFF7A0FE02E02020FFF738FE0A4B93F896
S31508001A804330012B02D11020FFF730FE064BB3F985
S31508001A904410002906DD1846012380F84330033038
S31508001AA0FFF770FF08BD00BF4409002008B5074BC3
S31508001AB0044613B10021AFF30080054B1868836A0A
S31508001AC003B19847204600F033F800BF0000000035
S31508001AD0B41C000870B50E4B0E4CE41AA410002571
S31508001AE01E46A54204D056F8253098470135F8E732
S31508001AF000F020F8084C094BE41AA41000251E46ED
S31508001B00A54204D056F8253098470135F8E770BD48
S31508001B1064000020640000206800002064000020A3
S31508001B2002440346934202D003F8011BFAE77047C2
S31508001B30FEE70000F8B500BFF8BC08BC9E46704733
S31508001B40F8B500BFF8BC08BC9E4670472E2E5C6CE4
S31508001B5069625C786D636C69625C7372635C786DEC
S31508001B6063345F6770696F2E630000004846005053
S31508001B7054460050604600506C46005014440050CD
S31508001B80204400502C440050384400502E2E5C6CE3
S31508001B9069625C786D636C69625C7372635C786DAC
S31508001BA0635F6770696F2E63000000002E2E5C6C01
S31508001BB069625C786D636C69625C7372635C786D8C
S31508001BC0635F757369632E63000000000040000CB4
S31508001BD000400000010000000080000C00400000EA
S31508001BE00200000000C0000C0040000003000000D6
S31508001BF00000010C00400000040000000040010C39
S31508001C0000400000050000000080010C00400000B4
S31508001C100600000000C0010C00400000070000009C
S31508001C200000020C00000200080000000000040C7E
S31508001C3000000400090000000000080C0000040071
S31508001C400A00000000000C0C000004000B00000055
S31508001C500000100C000004000C0000000000140C2A
S31508001C60000004000D0000000000180C000004002D
S31508001C700E00000000001C0C000004000F0000000D
S31508001C802E2E5C2E2E5C2E2E5C2E2E5C536F7572BD
S31508001C9063655C41524D434D345F584D43345C7522
S31508001CA06172742E630000004F70656E424C5400DA
S31108001CB0430000000400002000000000B3
S30D08001CBCA0E5FF7F010000000E
S31508001CC404000000000000000000000000000000FE
S31508001CD400000000000000000000000000000000F2
S31508001CE400000000B01C000800000000000000000E
S31508001CF400000000000000000000000000000000D2
S31508001D0400000000000000000000000000000000C1
S31508001D1400000000000000000000000000000000B1
S31108001D240000000025020008010200086B
S31508001D300000000000000000000000000000000095
S30908001D400000000091
S70508000000F2
